 redefineCFLH

 Timestamp is 7f0bac7b (reproducible build file hash)

 Preferred load address is 0000000180000000

 Start         Length     Name                   Class
 0001:00000000 00002cf0H .text$mn                CODE
 0001:00002cf0 00000036H .text$mn$00             CODE
 0001:00002d26 00000092H .text$x                 CODE
 0002:00000000 00000198H .idata$5                DATA
 0002:00000198 00000038H .00cfg                  DATA
 0002:000001d0 00000008H .CRT$XCA                DATA
 0002:000001d8 00000008H .CRT$XCZ                DATA
 0002:000001e0 00000008H .CRT$XIA                DATA
 0002:000001e8 00000008H .CRT$XIC                DATA
 0002:000001f0 00000008H .CRT$XIZ                DATA
 0002:000001f8 00000008H .CRT$XLA                DATA
 0002:00000200 00000008H .CRT$XLZ                DATA
 0002:00000208 00000008H .CRT$XPA                DATA
 0002:00000210 00000008H .CRT$XPZ                DATA
 0002:00000218 00000008H .CRT$XTA                DATA
 0002:00000220 00000010H .CRT$XTZ                DATA
 0002:00000228 00000000H .gehcont$y              DATA
 0002:00000228 00000000H .gfids$y                DATA
 0002:00000230 00001dd0H .rdata                  DATA
 0002:00002000 00000000H .rdata$CastGuardVftablesA DATA
 0002:00002000 00000000H .rdata$CastGuardVftablesC DATA
 0002:00002000 00000028H .rdata$T                DATA
 0002:00002028 000000b0H .rdata$voltmd           DATA
 0002:000020d8 00000320H .rdata$zzzdbg           DATA
 0002:000023f8 00000008H .rtc$IAA                DATA
 0002:00002400 00000008H .rtc$IZZ                DATA
 0002:00002408 00000008H .rtc$TAA                DATA
 0002:00002410 00000008H .rtc$TZZ                DATA
 0002:00002418 00000004H .tls                    DATA
 0002:0000241c 00000004H .tls$                   DATA
 0002:00002420 00000008H .tls$ZZZ                DATA
 0002:00002428 000002e8H .xdata                  DATA
 0002:00002710 000003f8H .edata                  DATA
 0002:00002b08 00000064H .idata$2                DATA
 0002:00002b6c 00000014H .idata$3                DATA
 0002:00002b80 00000198H .idata$4                DATA
 0002:00002d18 0000041eH .idata$6                DATA
 0003:00000000 00000080H .data                   DATA
 0003:00000080 0001b378H .bss                    DATA
 0004:00000000 00000384H .pdata                  DATA

  Address         Publics by Value              Rva+Base               Lib:Object

 0000:00000000       __AbsoluteZero             0000000000000000     <absolute>
 0000:00000000       ___safe_se_handler_count   0000000000000000     <absolute>
 0000:00000000       ___safe_se_handler_table   0000000000000000     <absolute>
 0000:00000000       __arm64x_extra_rfe_table   0000000000000000     <absolute>
 0000:00000000       __arm64x_extra_rfe_table_size 0000000000000000     <absolute>
 0000:00000000       __arm64x_native_entrypoint 0000000000000000     <absolute>
 0000:00000000       __arm64x_redirection_metadata 0000000000000000     <absolute>
 0000:00000000       __arm64x_redirection_metadata_count 0000000000000000     <absolute>
 0000:00000000       __dynamic_value_reloc_table 0000000000000000     <absolute>
 0000:00000000       __enclave_config           0000000000000000     <absolute>
 0000:00000000       __guard_check_icall_a64n_fptr 0000000000000000     <absolute>
 0000:00000000       __guard_eh_cont_count      0000000000000000     <absolute>
 0000:00000000       __guard_eh_cont_table      0000000000000000     <absolute>
 0000:00000000       __guard_fids_count         0000000000000000     <absolute>
 0000:00000000       __guard_fids_table         0000000000000000     <absolute>
 0000:00000000       __guard_iat_count          0000000000000000     <absolute>
 0000:00000000       __guard_iat_table          0000000000000000     <absolute>
 0000:00000000       __guard_longjmp_count      0000000000000000     <absolute>
 0000:00000000       __guard_longjmp_table      0000000000000000     <absolute>
 0000:00000000       __hybrid_auxiliary_iat     0000000000000000     <absolute>
 0000:00000000       __hybrid_auxiliary_iat_copy 0000000000000000     <absolute>
 0000:00000000       __hybrid_code_map          0000000000000000     <absolute>
 0000:00000000       __hybrid_code_map_count    0000000000000000     <absolute>
 0000:00000000       __x64_code_ranges_to_entry_points 0000000000000000     <absolute>
 0000:00000000       __x64_code_ranges_to_entry_points_count 0000000000000000     <absolute>
 0000:00000100       __guard_flags              0000000000000100     <absolute>
 0000:00000000       __ImageBase                0000000180000000     <linker-defined>
 0001:00000000       ?NewObject@JNIEnv_@@QEAAPEAV_jobject@@PEAV_jclass@@PEAU_jmethodID@@ZZ 0000000180001000 f i libredefineCFLH.obj
 0001:00000024       ?SetEventNotificationMode@_jvmtiEnv@@QEAA?AW4jvmtiError@@W4jvmtiEventMode@@W4jvmtiEvent@@PEAV_jobject@@ZZ 0000000180001024 f i libredefineCFLH.obj
 0001:0000002c       ?TranslateError@@YAPEBDW4jvmtiError@@@Z 000000018000102c f   libredefineCFLH.obj
 0001:000002e4       ?nsk_jni_check_exception@@YAHPEAUJNIEnv_@@QEBDH@Z 00000001800012e4 f   libredefineCFLH.obj
 0001:00000428       ?nsk_jni_lverify@@YAHHPEAUJNIEnv_@@HQEBDH1ZZ 0000000180001428 f   libredefineCFLH.obj
 0001:000004c8       Agent_Initialize           00000001800014c8 f   libredefineCFLH.obj
 0001:000006bc       Agent_OnAttach             00000001800016bc f   libredefineCFLH.obj
 0001:000006bc       Agent_OnLoad               00000001800016bc f   libredefineCFLH.obj
 0001:000006c4       ClassFileLoadHook          00000001800016c4 f   libredefineCFLH.obj
 0001:00000800       Java_nsk_jvmti_unit_FollowReferences_FollowRefObjects_addRefToVerify 0000000180001800 f   libredefineCFLH.obj
 0001:000009bc       Java_nsk_jvmti_unit_FollowReferences_FollowRefObjects_getTag 00000001800019bc f   libredefineCFLH.obj
 0001:00000a78       Java_nsk_jvmti_unit_FollowReferences_FollowRefObjects_resetRefsToVerify 0000000180001a78 f   libredefineCFLH.obj
 0001:00000a80       Java_nsk_jvmti_unit_FollowReferences_FollowRefObjects_resetTags 0000000180001a80 f   libredefineCFLH.obj
 0001:00000ac4       Java_nsk_jvmti_unit_FollowReferences_FollowRefObjects_setTag 0000000180001ac4 f   libredefineCFLH.obj
 0001:00000d10       Java_nsk_jvmti_unit_events_redefineCFLH_JvmtiTest_GetResult 0000000180001d10 f   libredefineCFLH.obj
 0001:00000d18       Java_nsk_jvmti_unit_events_redefineCFLH_JvmtiTest_makeRedefinition 0000000180001d18 f   libredefineCFLH.obj
 0001:00000e20       Java_nsk_share_jvmti_ArgumentHandler_getAgentOptionsString 0000000180001e20 f   libredefineCFLH.obj
 0001:00000ecc       Java_nsk_share_jvmti_DebugeeClass_checkStatus 0000000180001ecc f   libredefineCFLH.obj
 0001:00000f54       Java_nsk_share_jvmti_DebugeeClass_resetAgentData 0000000180001f54 f   libredefineCFLH.obj
 0001:00000fb4       Java_nsk_share_jvmti_RedefineAgent_agentStatus 0000000180001fb4 f   libredefineCFLH.obj
 0001:00000fc0       Java_nsk_share_jvmti_RedefineAgent_isRedefined 0000000180001fc0 f   libredefineCFLH.obj
 0001:00000fcc       Java_nsk_share_jvmti_RedefineAgent_redefineAttempted 0000000180001fcc f   libredefineCFLH.obj
 0001:00000fd8       MA_checkStatus             0000000180001fd8 f   libredefineCFLH.obj
 0001:0000107c       VMInit                     000000018000207c f   libredefineCFLH.obj
 0001:0000109c       __local_stdio_printf_options 000000018000209c f i libredefineCFLH.obj
 0001:0000126c       exitOnError                000000018000226c f   libredefineCFLH.obj
 0001:00001320       fprintf                    0000000180002320 f i libredefineCFLH.obj
 0001:00001364       nsk_jvmti_lverify          0000000180002364 f   libredefineCFLH.obj
 0001:00001454       nsk_jvmti_resetAgentData   0000000180002454 f   libredefineCFLH.obj
 0001:000014c8       nsk_lcomplain              00000001800024c8 f   libredefineCFLH.obj
 0001:000014e8       nsk_ldisplay               00000001800024e8 f   libredefineCFLH.obj
 0001:00001508       nsk_ltrace                 0000000180002508 f   libredefineCFLH.obj
 0001:00001528       nsk_lvcomplain             0000000180002528 f   libredefineCFLH.obj
 0001:000016e0       nsk_lvdisplay              00000001800026e0 f   libredefineCFLH.obj
 0001:0000172c       nsk_lverify                000000018000272c f   libredefineCFLH.obj
 0001:00001788       nsk_lvtrace                0000000180002788 f   libredefineCFLH.obj
 0001:000017e8       nsk_printf                 00000001800027e8 f   libredefineCFLH.obj
 0001:00001810       nsk_vprintf                0000000180002810 f   libredefineCFLH.obj
 0001:000018c4       printf                     00000001800028c4 f i libredefineCFLH.obj
 0001:00001dc4       __raise_securityfailure    0000000180002dc4 f   MSVCRT:gs_report.obj
 0001:00001df8       __report_gsfailure         0000000180002df8 f   MSVCRT:gs_report.obj
 0001:00002038       __GSHandlerCheck           0000000180003038 f   MSVCRT:gshandler.obj
 0001:00002058       __GSHandlerCheckCommon     0000000180003058 f   MSVCRT:gshandler.obj
 0001:000020d0       __security_check_cookie    00000001800030d0 f   MSVCRT:amdsecgs.obj
 0001:00002410       _DllMainCRTStartup         0000000180003410 f   MSVCRT:dll_dllmain.obj
 0001:00002450       __scrt_acquire_startup_lock 0000000180003450 f   MSVCRT:utility.obj
 0001:0000248c       __scrt_dllmain_after_initialize_c 000000018000348c f   MSVCRT:utility.obj
 0001:000024c0       __scrt_dllmain_before_initialize_c 00000001800034c0 f   MSVCRT:utility.obj
 0001:000024d8       __scrt_dllmain_crt_thread_attach 00000001800034d8 f   MSVCRT:utility.obj
 0001:00002500       __scrt_dllmain_crt_thread_detach 0000000180003500 f   MSVCRT:utility.obj
 0001:00002518       __scrt_dllmain_exception_filter 0000000180003518 f   MSVCRT:utility.obj
 0001:00002578       __scrt_dllmain_uninitialize_c 0000000180003578 f   MSVCRT:utility.obj
 0001:000025a8       __scrt_dllmain_uninitialize_critical 00000001800035a8 f   MSVCRT:utility.obj
 0001:000025bc       __scrt_initialize_crt      00000001800035bc f   MSVCRT:utility.obj
 0001:00002608       __scrt_initialize_onexit_tables 0000000180003608 f   MSVCRT:utility.obj
 0001:00002694       __scrt_is_nonwritable_in_current_image 0000000180003694 f   MSVCRT:utility.obj
 0001:0000272c       __scrt_release_startup_lock 000000018000372c f   MSVCRT:utility.obj
 0001:00002750       __scrt_uninitialize_crt    0000000180003750 f   MSVCRT:utility.obj
 0001:0000277c       _onexit                    000000018000377c f   MSVCRT:utility.obj
 0001:000027b8       atexit                     00000001800037b8 f   MSVCRT:utility.obj
 0001:000027d0       __crt_debugger_hook        00000001800037d0 f   MSVCRT:utility_desktop.obj
 0001:000027d8       __scrt_fastfail            00000001800037d8 f   MSVCRT:utility_desktop.obj
 0001:00002924       _guard_check_icall_nop     0000000180003924 f i MSVCRT:guard_support.obj
 0001:00002928       __security_init_cookie     0000000180003928 f   MSVCRT:gs_support.obj
 0001:000029d4       DllMain                    00000001800039d4 f   MSVCRT:dll_dllmain_stub.obj
 0001:000029f8       ?__scrt_initialize_type_info@@YAXXZ 00000001800039f8 f   MSVCRT:tncleanup.obj
 0001:00002a08       ?__scrt_uninitialize_type_info@@YAXXZ 0000000180003a08 f   MSVCRT:tncleanup.obj
 0001:00002a14       __local_stdio_scanf_options 0000000180003a14 f i MSVCRT:default_local_stdio_options.obj
 0001:00002a1c       __scrt_initialize_default_local_stdio_options 0000000180003a1c f   MSVCRT:default_local_stdio_options.obj
 0001:00002a38       __scrt_get_dyn_tls_init_callback 0000000180003a38 f   MSVCRT:dyn_tls_init.obj
 0001:00002a40       _RTC_Initialize            0000000180003a40 f   MSVCRT:initsect.obj
 0001:00002a7c       _RTC_Terminate             0000000180003a7c f   MSVCRT:initsect.obj
 0001:00002ab8       __isa_available_init       0000000180003ab8 f   MSVCRT:cpu_disp.obj
 0001:00002c64       _get_startup_argv_mode     0000000180003c64 f   MSVCRT:argv_mode.obj
 0001:00002c6c       __scrt_is_ucrt_dll_in_use  0000000180003c6c f   MSVCRT:ucrt_detection.obj
 0001:00002c80       memcpy                     0000000180003c80 f   vcruntime:VCRUNTIME140.dll
 0001:00002c86       memset                     0000000180003c86 f   vcruntime:VCRUNTIME140.dll
 0001:00002c8c       strchr                     0000000180003c8c f   vcruntime:VCRUNTIME140.dll
 0001:00002c92       __C_specific_handler       0000000180003c92 f   vcruntime:VCRUNTIME140.dll
 0001:00002c98       __std_type_info_destroy_list 0000000180003c98 f   vcruntime:VCRUNTIME140.dll
 0001:00002c9e       strcmp                     0000000180003c9e f   ucrt:api-ms-win-crt-string-l1-1-0.dll
 0001:00002ca4       strlen                     0000000180003ca4 f   ucrt:api-ms-win-crt-string-l1-1-0.dll
 0001:00002caa       _initterm                  0000000180003caa f   ucrt:api-ms-win-crt-runtime-l1-1-0.dll
 0001:00002cb0       _initterm_e                0000000180003cb0 f   ucrt:api-ms-win-crt-runtime-l1-1-0.dll
 0001:00002cb6       _seh_filter_dll            0000000180003cb6 f   ucrt:api-ms-win-crt-runtime-l1-1-0.dll
 0001:00002cbc       _configure_narrow_argv     0000000180003cbc f   ucrt:api-ms-win-crt-runtime-l1-1-0.dll
 0001:00002cc2       _initialize_narrow_environment 0000000180003cc2 f   ucrt:api-ms-win-crt-runtime-l1-1-0.dll
 0001:00002cc8       _initialize_onexit_table   0000000180003cc8 f   ucrt:api-ms-win-crt-runtime-l1-1-0.dll
 0001:00002cce       _register_onexit_function  0000000180003cce f   ucrt:api-ms-win-crt-runtime-l1-1-0.dll
 0001:00002cd4       _execute_onexit_table      0000000180003cd4 f   ucrt:api-ms-win-crt-runtime-l1-1-0.dll
 0001:00002cda       _crt_atexit                0000000180003cda f   ucrt:api-ms-win-crt-runtime-l1-1-0.dll
 0001:00002ce0       _cexit                     0000000180003ce0 f   ucrt:api-ms-win-crt-runtime-l1-1-0.dll
 0001:00002ce8       __acrt_initialize          0000000180003ce8 f   MSVCRT:ucrt_stubs.obj
 0001:00002ce8       __acrt_thread_attach       0000000180003ce8 f   MSVCRT:ucrt_stubs.obj
 0001:00002ce8       __acrt_thread_detach       0000000180003ce8 f   MSVCRT:ucrt_stubs.obj
 0001:00002ce8       __acrt_uninitialize        0000000180003ce8 f   MSVCRT:ucrt_stubs.obj
 0001:00002ce8       __acrt_uninitialize_critical 0000000180003ce8 f   MSVCRT:ucrt_stubs.obj
 0001:00002ce8       __scrt_stub_for_acrt_initialize 0000000180003ce8 f   MSVCRT:ucrt_stubs.obj
 0001:00002ce8       __scrt_stub_for_acrt_thread_attach 0000000180003ce8 f   MSVCRT:ucrt_stubs.obj
 0001:00002ce8       __scrt_stub_for_acrt_thread_detach 0000000180003ce8 f   MSVCRT:ucrt_stubs.obj
 0001:00002ce8       __scrt_stub_for_acrt_uninitialize 0000000180003ce8 f   MSVCRT:ucrt_stubs.obj
 0001:00002ce8       __scrt_stub_for_acrt_uninitialize_critical 0000000180003ce8 f   MSVCRT:ucrt_stubs.obj
 0001:00002ce8       __vcrt_initialize          0000000180003ce8 f   MSVCRT:ucrt_stubs.obj
 0001:00002ce8       __vcrt_thread_attach       0000000180003ce8 f   MSVCRT:ucrt_stubs.obj
 0001:00002ce8       __vcrt_thread_detach       0000000180003ce8 f   MSVCRT:ucrt_stubs.obj
 0001:00002ce8       __vcrt_uninitialize        0000000180003ce8 f   MSVCRT:ucrt_stubs.obj
 0001:00002ce8       __vcrt_uninitialize_critical 0000000180003ce8 f   MSVCRT:ucrt_stubs.obj
 0001:00002cec       __scrt_stub_for_is_c_termination_complete 0000000180003cec f   MSVCRT:ucrt_stubs.obj
 0001:00002cec       _is_c_termination_complete 0000000180003cec f   MSVCRT:ucrt_stubs.obj
 0001:00002d00       _guard_dispatch_icall_nop  0000000180003d00 f   MSVCRT:guard_dispatch.obj
 0001:00002d20       _guard_xfg_dispatch_icall_nop 0000000180003d20 f   MSVCRT:guard_xfg_dispatch.obj
 0002:00000000       __imp_RtlCaptureContext    0000000180004000     kernel32:KERNEL32.dll
 0002:00000008       __imp_RtlLookupFunctionEntry 0000000180004008     kernel32:KERNEL32.dll
 0002:00000010       __imp_RtlVirtualUnwind     0000000180004010     kernel32:KERNEL32.dll
 0002:00000018       __imp_UnhandledExceptionFilter 0000000180004018     kernel32:KERNEL32.dll
 0002:00000020       __imp_SetUnhandledExceptionFilter 0000000180004020     kernel32:KERNEL32.dll
 0002:00000028       __imp_GetCurrentProcess    0000000180004028     kernel32:KERNEL32.dll
 0002:00000030       __imp_TerminateProcess     0000000180004030     kernel32:KERNEL32.dll
 0002:00000038       __imp_IsProcessorFeaturePresent 0000000180004038     kernel32:KERNEL32.dll
 0002:00000040       __imp_CloseHandle          0000000180004040     kernel32:KERNEL32.dll
 0002:00000048       __imp_InitializeCriticalSectionAndSpinCount 0000000180004048     kernel32:KERNEL32.dll
 0002:00000050       __imp_DeleteCriticalSection 0000000180004050     kernel32:KERNEL32.dll
 0002:00000058       __imp_CreateEventW         0000000180004058     kernel32:KERNEL32.dll
 0002:00000060       __imp_GetModuleHandleW     0000000180004060     kernel32:KERNEL32.dll
 0002:00000068       __imp_GetProcAddress       0000000180004068     kernel32:KERNEL32.dll
 0002:00000070       __imp_IsDebuggerPresent    0000000180004070     kernel32:KERNEL32.dll
 0002:00000078       __imp_QueryPerformanceCounter 0000000180004078     kernel32:KERNEL32.dll
 0002:00000080       __imp_GetCurrentProcessId  0000000180004080     kernel32:KERNEL32.dll
 0002:00000088       __imp_GetCurrentThreadId   0000000180004088     kernel32:KERNEL32.dll
 0002:00000090       __imp_GetSystemTimeAsFileTime 0000000180004090     kernel32:KERNEL32.dll
 0002:00000098       __imp_DisableThreadLibraryCalls 0000000180004098     kernel32:KERNEL32.dll
 0002:000000a0       __imp_InitializeSListHead  00000001800040a0     kernel32:KERNEL32.dll
 0002:000000a8       \177KERNEL32_NULL_THUNK_DATA 00000001800040a8     kernel32:KERNEL32.dll
 0002:000000b0       __imp_memcpy               00000001800040b0     vcruntime:VCRUNTIME140.dll
 0002:000000b8       __imp_memset               00000001800040b8     vcruntime:VCRUNTIME140.dll
 0002:000000c0       __imp_strchr               00000001800040c0     vcruntime:VCRUNTIME140.dll
 0002:000000c8       __imp___C_specific_handler 00000001800040c8     vcruntime:VCRUNTIME140.dll
 0002:000000d0       __imp___std_type_info_destroy_list 00000001800040d0     vcruntime:VCRUNTIME140.dll
 0002:000000d8       \177VCRUNTIME140_NULL_THUNK_DATA 00000001800040d8     vcruntime:VCRUNTIME140.dll
 0002:000000e0       __imp__errno               00000001800040e0     ucrt:api-ms-win-crt-runtime-l1-1-0.dll
 0002:000000e8       __imp_exit                 00000001800040e8     ucrt:api-ms-win-crt-runtime-l1-1-0.dll
 0002:000000f0       __imp__cexit               00000001800040f0     ucrt:api-ms-win-crt-runtime-l1-1-0.dll
 0002:000000f8       __imp__crt_atexit          00000001800040f8     ucrt:api-ms-win-crt-runtime-l1-1-0.dll
 0002:00000100       __imp__execute_onexit_table 0000000180004100     ucrt:api-ms-win-crt-runtime-l1-1-0.dll
 0002:00000108       __imp__register_onexit_function 0000000180004108     ucrt:api-ms-win-crt-runtime-l1-1-0.dll
 0002:00000110       __imp__initialize_onexit_table 0000000180004110     ucrt:api-ms-win-crt-runtime-l1-1-0.dll
 0002:00000118       __imp__initialize_narrow_environment 0000000180004118     ucrt:api-ms-win-crt-runtime-l1-1-0.dll
 0002:00000120       __imp__configure_narrow_argv 0000000180004120     ucrt:api-ms-win-crt-runtime-l1-1-0.dll
 0002:00000128       __imp__seh_filter_dll      0000000180004128     ucrt:api-ms-win-crt-runtime-l1-1-0.dll
 0002:00000130       __imp__initterm_e          0000000180004130     ucrt:api-ms-win-crt-runtime-l1-1-0.dll
 0002:00000138       __imp__initterm            0000000180004138     ucrt:api-ms-win-crt-runtime-l1-1-0.dll
 0002:00000140       \177api-ms-win-crt-runtime-l1-1-0_NULL_THUNK_DATA 0000000180004140     ucrt:api-ms-win-crt-runtime-l1-1-0.dll
 0002:00000148       __imp___acrt_iob_func      0000000180004148     ucrt:api-ms-win-crt-stdio-l1-1-0.dll
 0002:00000150       __imp_fflush               0000000180004150     ucrt:api-ms-win-crt-stdio-l1-1-0.dll
 0002:00000158       __imp___stdio_common_vsprintf 0000000180004158     ucrt:api-ms-win-crt-stdio-l1-1-0.dll
 0002:00000160       __imp___stdio_common_vfprintf 0000000180004160     ucrt:api-ms-win-crt-stdio-l1-1-0.dll
 0002:00000168       \177api-ms-win-crt-stdio-l1-1-0_NULL_THUNK_DATA 0000000180004168     ucrt:api-ms-win-crt-stdio-l1-1-0.dll
 0002:00000170       __imp_strcmp               0000000180004170     ucrt:api-ms-win-crt-string-l1-1-0.dll
 0002:00000178       __imp__strdup              0000000180004178     ucrt:api-ms-win-crt-string-l1-1-0.dll
 0002:00000178       __imp_strdup               0000000180004178     ucrt:api-ms-win-crt-string-l1-1-0.dll
 0002:00000180       __imp_strlen               0000000180004180     ucrt:api-ms-win-crt-string-l1-1-0.dll
 0002:00000188       __imp_strncpy              0000000180004188     ucrt:api-ms-win-crt-string-l1-1-0.dll
 0002:00000190       \177api-ms-win-crt-string-l1-1-0_NULL_THUNK_DATA 0000000180004190     ucrt:api-ms-win-crt-string-l1-1-0.dll
 0002:00000198       __guard_check_icall_fptr   0000000180004198     MSVCRT:guard_support.obj
 0002:000001a0       __guard_xfg_check_icall_fptr 00000001800041a0     MSVCRT:guard_support.obj
 0002:000001a8       __guard_dispatch_icall_fptr 00000001800041a8     MSVCRT:guard_support.obj
 0002:000001b0       __guard_xfg_dispatch_icall_fptr 00000001800041b0     MSVCRT:guard_support.obj
 0002:000001b8       __guard_xfg_table_dispatch_icall_fptr 00000001800041b8     MSVCRT:guard_support.obj
 0002:000001c0       __castguard_check_failure_os_handled_fptr 00000001800041c0     MSVCRT:guard_support.obj
 0002:000001c8       __guard_memcpy_fptr        00000001800041c8     vcruntime:softmemtag.obj
 0002:000001d0       __xc_a                     00000001800041d0     MSVCRT:initializers.obj
 0002:000001d8       __xc_z                     00000001800041d8     MSVCRT:initializers.obj
 0002:000001e0       __xi_a                     00000001800041e0     MSVCRT:initializers.obj
 0002:000001f0       __xi_z                     00000001800041f0     MSVCRT:initializers.obj
 0002:000001f8       __xl_a                     00000001800041f8     MSVCRT:tlssup.obj
 0002:00000200       __xl_z                     0000000180004200     MSVCRT:tlssup.obj
 0002:00000208       __xp_a                     0000000180004208     MSVCRT:initializers.obj
 0002:00000210       __xp_z                     0000000180004210     MSVCRT:initializers.obj
 0002:00000218       __xt_a                     0000000180004218     MSVCRT:initializers.obj
 0002:00000220       __xt_z                     0000000180004220     MSVCRT:initializers.obj
 0002:00000230       g_refKindStr               0000000180004230     libredefineCFLH.obj
 0002:000003e0       ??_C@_09BPLDFGCI@unknown_0@ 00000001800043e0     libredefineCFLH.obj
 0002:000003f0       ??_C@_0BL@FPNMECJD@JVMTI_HEAP_REFERENCE_CLASS@ 00000001800043f0     libredefineCFLH.obj
 0002:00000410       ??_C@_0BL@FKGKKLNM@JVMTI_HEAP_REFERENCE_FIELD@ 0000000180004410     libredefineCFLH.obj
 0002:00000430       ??_C@_0CD@CAEHCFJF@JVMTI_HEAP_REFERENCE_ARRAY_ELEM@ 0000000180004430     libredefineCFLH.obj
 0002:00000458       ??_C@_0CC@DNEBMCNK@JVMTI_HEAP_REFERENCE_CLASS_LOAD@ 0000000180004458     libredefineCFLH.obj
 0002:00000480       ??_C@_0BN@CJMIPEBB@JVMTI_HEAP_REFERENCE_SIGNERS@ 0000000180004480     libredefineCFLH.obj
 0002:000004a0       ??_C@_0CH@HBOIDPEB@JVMTI_HEAP_REFERENCE_PROTECTION@ 00000001800044a0     libredefineCFLH.obj
 0002:000004c8       ??_C@_0BP@MDKGDGKL@JVMTI_HEAP_REFERENCE_INTERFACE@ 00000001800044c8     libredefineCFLH.obj
 0002:000004e8       ??_C@_0CC@JJMIHNJH@JVMTI_HEAP_REFERENCE_STATIC_FIE@ 00000001800044e8     libredefineCFLH.obj
 0002:00000510       ??_C@_0CD@IDHEEGID@JVMTI_HEAP_REFERENCE_CONSTANT_P@ 0000000180004510     libredefineCFLH.obj
 0002:00000538       ??_C@_0CA@EFFCHNG@JVMTI_HEAP_REFERENCE_SUPERCLASS@ 0000000180004538     libredefineCFLH.obj
 0002:00000558       ??_C@_0L@PCDFHGCJ@unknown_11@ 0000000180004558     libredefineCFLH.obj
 0002:00000568       ??_C@_0L@NJBICFOK@unknown_12@ 0000000180004568     libredefineCFLH.obj
 0002:00000578       ??_C@_0L@MAADBEKL@unknown_13@ 0000000180004578     libredefineCFLH.obj
 0002:00000588       ??_C@_0L@IPECICGM@unknown_14@ 0000000180004588     libredefineCFLH.obj
 0002:00000598       ??_C@_0L@JGFJLDCN@unknown_15@ 0000000180004598     libredefineCFLH.obj
 0002:000005a8       ??_C@_0L@LNHEOAOO@unknown_16@ 00000001800045a8     libredefineCFLH.obj
 0002:000005b8       ??_C@_0L@KEGPNBKP@unknown_17@ 00000001800045b8     libredefineCFLH.obj
 0002:000005c8       ??_C@_0L@CDPHMNGA@unknown_18@ 00000001800045c8     libredefineCFLH.obj
 0002:000005d8       ??_C@_0L@DKOMPMCB@unknown_19@ 00000001800045d8     libredefineCFLH.obj
 0002:000005e8       ??_C@_0L@OJGIPJDB@unknown_20@ 00000001800045e8     libredefineCFLH.obj
 0002:000005f8       ??_C@_0CA@KAOFNDEM@JVMTI_HEAP_REFERENCE_JNI_GLOBAL@ 00000001800045f8     libredefineCFLH.obj
 0002:00000618       ??_C@_0CC@HPFAJBK@JVMTI_HEAP_REFERENCE_SYSTEM_CLA@ 0000000180004618     libredefineCFLH.obj
 0002:00000640       ??_C@_0BN@FDEGFOHC@JVMTI_HEAP_REFERENCE_MONITOR@ 0000000180004640     libredefineCFLH.obj
 0002:00000660       ??_C@_0CB@HKIBCMAJ@JVMTI_HEAP_REFERENCE_STACK_LOCA@ 0000000180004660     libredefineCFLH.obj
 0002:00000688       ??_C@_0BP@EAACMMOE@JVMTI_HEAP_REFERENCE_JNI_LOCAL@ 0000000180004688     libredefineCFLH.obj
 0002:000006a8       ??_C@_0BM@IJDEOGOE@JVMTI_HEAP_REFERENCE_THREAD@ 00000001800046a8     libredefineCFLH.obj
 0002:000006c8       ??_C@_0BL@EDGPPKC@JVMTI_HEAP_REFERENCE_OTHER@ 00000001800046c8     libredefineCFLH.obj
 0002:000006e4       ??_C@_04BCJPDBDA@Code@     00000001800046e4     libredefineCFLH.obj
 0002:000006f0       ??_C@_0BA@OCLMCFKC@LineNumberTable@ 00000001800046f0     libredefineCFLH.obj
 0002:00000700       ??_C@_0BD@CPAEPILC@LocalVariableTable@ 0000000180004700     libredefineCFLH.obj
 0002:00000718       ??_C@_0BH@NMBDNHBD@LocalVariableTypeTable@ 0000000180004718     libredefineCFLH.obj
 0002:00000730       ??_C@_0O@HIHEEDNJ@StackMapTable@ 0000000180004730     libredefineCFLH.obj
 0002:00000740       ??_C@_0CO@MLEIEIFA@nsk?1jvmti?1unit?1events?1redefineC@ 0000000180004740     libredefineCFLH.obj
 0002:00000770       ??_C@_0L@HCDIAMJG@?9?5?$CFs?0?5?$CFd?3?5@ 0000000180004770     libredefineCFLH.obj
 0002:00000780       ??_C@_0JI@HLPECLFI@?$CD?5?4?4?4?6?$CD?5ERROR?3?5too?5many?5complai@ 0000000180004780     libredefineCFLH.obj
 0002:00000820       ??_C@_0ED@JNEKCCOB@The?5following?5fake?5exception?5st@ 0000000180004820     libredefineCFLH.obj
 0002:00000868       ??_C@_0CN@FCNMDFBH@nsk?4share?4Fake_Exception_for_RU@ 0000000180004868     libredefineCFLH.obj
 0002:00000898       ??_C@_08PGFFNAEI@?$CI?$CFs?3?$CFd?$CJ?5@ 0000000180004898     libredefineCFLH.obj
 0002:000008a8       ??_C@_0DP@IENMAEGI@s?2test?2hotspot?2jtreg?2vmTestbase@ 00000001800048a8     libredefineCFLH.obj
 0002:000008e8       ??_C@_0BL@NDJLFFJB@?7at?5nsk_lvcomplain?$CI?$CFs?3?$CFd?$CJ?6@ 00000001800048e8     libredefineCFLH.obj
 0002:00000908       ??_C@_0BC@JOOKAFKF@?$CD?5ERROR?3?5?$CFs?0?5?$CFd?3?5@ 0000000180004908     libredefineCFLH.obj
 0002:00000920       ??_C@_09KJEAHMEH@?$CD?5ERROR?3?5@ 0000000180004920     libredefineCFLH.obj
 0002:0000092c       ??_C@_02GPIOPFAK@?$DO?$DO@ 000000018000492c     libredefineCFLH.obj
 0002:00000930       ??_C@_02FODMEDOG@?$DM?$DM@ 0000000180004930     libredefineCFLH.obj
 0002:00000934       ??_C@_02DJGKEECL@?4?4@     0000000180004934     libredefineCFLH.obj
 0002:00000938       ??_C@_0O@CJPGJOAF@?9?5?$CFs?0?5?$CFd?3?5?$CFs?5@ 0000000180004938     libredefineCFLH.obj
 0002:00000948       ??_C@_0CB@IAKPDOIC@?$CD?5?5?5verified?5assertion?5is?5FALSE@ 0000000180004948     libredefineCFLH.obj
 0002:00000970       ??_C@_0CO@LGONDEPD@stdout?3?5fflush?5failed?5?9?5err?$DN?$CFd?5@ 0000000180004970     libredefineCFLH.obj
 0002:000009a0       ??_C@_0CO@KBGKJPBD@stderr?3?5fflush?5failed?5?9?5err?$DN?$CFd?5@ 00000001800049a0     libredefineCFLH.obj
 0002:000009d0       ??_C@_0BB@JCNMKLLK@JVMTI_ERROR_NONE@ 00000001800049d0     libredefineCFLH.obj
 0002:000009e8       ??_C@_0BL@LDIMKLPH@JVMTI_ERROR_INVALID_THREAD@ 00000001800049e8     libredefineCFLH.obj
 0002:00000a08       ??_C@_0CB@PJFPAIKJ@JVMTI_ERROR_INVALID_THREAD_GROU@ 0000000180004a08     libredefineCFLH.obj
 0002:00000a30       ??_C@_0BN@LLMKHMNF@JVMTI_ERROR_INVALID_PRIORITY@ 0000000180004a30     libredefineCFLH.obj
 0002:00000a50       ??_C@_0CB@MBOFKAGB@JVMTI_ERROR_THREAD_NOT_SUSPENDE@ 0000000180004a50     libredefineCFLH.obj
 0002:00000a78       ??_C@_0BN@FABOLPBI@JVMTI_ERROR_THREAD_SUSPENDED@ 0000000180004a78     libredefineCFLH.obj
 0002:00000a98       ??_C@_0BN@FDGNOBJM@JVMTI_ERROR_THREAD_NOT_ALIVE@ 0000000180004a98     libredefineCFLH.obj
 0002:00000ab8       ??_C@_0BL@GOBIFKNJ@JVMTI_ERROR_INVALID_OBJECT@ 0000000180004ab8     libredefineCFLH.obj
 0002:00000ad8       ??_C@_0BK@FCMAJPPC@JVMTI_ERROR_INVALID_CLASS@ 0000000180004ad8     libredefineCFLH.obj
 0002:00000af8       ??_C@_0BP@IKLLBKEB@JVMTI_ERROR_CLASS_NOT_PREPARED@ 0000000180004af8     libredefineCFLH.obj
 0002:00000b18       ??_C@_0BN@KLPPLKG@JVMTI_ERROR_INVALID_METHODID@ 0000000180004b18     libredefineCFLH.obj
 0002:00000b38       ??_C@_0BN@BCEKOKND@JVMTI_ERROR_INVALID_LOCATION@ 0000000180004b38     libredefineCFLH.obj
 0002:00000b58       ??_C@_0BM@DFDGPME@JVMTI_ERROR_INVALID_FIELDID@ 0000000180004b58     libredefineCFLH.obj
 0002:00000b78       ??_C@_0BL@NELIEPEC@JVMTI_ERROR_NO_MORE_FRAMES@ 0000000180004b78     libredefineCFLH.obj
 0002:00000b98       ??_C@_0BJ@BDBECFDM@JVMTI_ERROR_OPAQUE_FRAME@ 0000000180004b98     libredefineCFLH.obj
 0002:00000bb8       ??_C@_0BK@MIIFNLOB@JVMTI_ERROR_TYPE_MISMATCH@ 0000000180004bb8     libredefineCFLH.obj
 0002:00000bd8       ??_C@_0BJ@HPCAOILC@JVMTI_ERROR_INVALID_SLOT@ 0000000180004bd8     libredefineCFLH.obj
 0002:00000bf8       ??_C@_0BG@CHILOPNI@JVMTI_ERROR_DUPLICATE@ 0000000180004bf8     libredefineCFLH.obj
 0002:00000c10       ??_C@_0BG@DIEMLHKM@JVMTI_ERROR_NOT_FOUND@ 0000000180004c10     libredefineCFLH.obj
 0002:00000c28       ??_C@_0BM@NHMCKHOB@JVMTI_ERROR_INVALID_MONITOR@ 0000000180004c28     libredefineCFLH.obj
 0002:00000c48       ??_C@_0BO@PPEDAJGL@JVMTI_ERROR_NOT_MONITOR_OWNER@ 0000000180004c48     libredefineCFLH.obj
 0002:00000c68       ??_C@_0BG@FCAIPEID@JVMTI_ERROR_INTERRUPT@ 0000000180004c68     libredefineCFLH.obj
 0002:00000c80       ??_C@_0CB@EGDBNKOI@JVMTI_ERROR_INVALID_CLASS_FORMA@ 0000000180004c80     libredefineCFLH.obj
 0002:00000ca8       ??_C@_0CG@DGKOGIAL@JVMTI_ERROR_CIRCULAR_CLASS_DEFI@ 0000000180004ca8     libredefineCFLH.obj
 0002:00000cd0       ??_C@_0BP@ICEALPKC@JVMTI_ERROR_FAILS_VERIFICATION@ 0000000180004cd0     libredefineCFLH.obj
 0002:00000cf0       ??_C@_0DC@JDACLMIO@JVMTI_ERROR_UNSUPPORTED_REDEFIN@ 0000000180004cf0     libredefineCFLH.obj
 0002:00000d28       ??_C@_0DE@GKDKNOMJ@JVMTI_ERROR_UNSUPPORTED_REDEFIN@ 0000000180004d28     libredefineCFLH.obj
 0002:00000d60       ??_C@_0BO@LAFKIOG@JVMTI_ERROR_INVALID_TYPESTATE@ 0000000180004d60     libredefineCFLH.obj
 0002:00000d80       ??_C@_0DH@INDGCLLB@JVMTI_ERROR_UNSUPPORTED_REDEFIN@ 0000000180004d80     libredefineCFLH.obj
 0002:00000db8       ??_C@_0DE@NHEOMMGI@JVMTI_ERROR_UNSUPPORTED_REDEFIN@ 0000000180004db8     libredefineCFLH.obj
 0002:00000df0       ??_C@_0CA@EKPNJOEP@JVMTI_ERROR_UNSUPPORTED_VERSION@ 0000000180004df0     libredefineCFLH.obj
 0002:00000e10       ??_C@_0BN@OFFMAHHL@JVMTI_ERROR_NAMES_DONT_MATCH@ 0000000180004e10     libredefineCFLH.obj
 0002:00000e30       ??_C@_0DN@HHBBLAKE@JVMTI_ERROR_UNSUPPORTED_REDEFIN@ 0000000180004e30     libredefineCFLH.obj
 0002:00000e70       ??_C@_0DO@HMBGBGNA@JVMTI_ERROR_UNSUPPORTED_REDEFIN@ 0000000180004e70     libredefineCFLH.obj
 0002:00000eb0       ??_C@_0BP@PBECGKHJ@JVMTI_ERROR_UNMODIFIABLE_CLASS@ 0000000180004eb0     libredefineCFLH.obj
 0002:00000ed0       ??_C@_0BK@CANILEHF@JVMTI_ERROR_NOT_AVAILABLE@ 0000000180004ed0     libredefineCFLH.obj
 0002:00000ef0       ??_C@_0CE@INJKMEFK@JVMTI_ERROR_MUST_POSSESS_CAPABI@ 0000000180004ef0     libredefineCFLH.obj
 0002:00000f18       ??_C@_0BJ@LBFPFPDM@JVMTI_ERROR_NULL_POINTER@ 0000000180004f18     libredefineCFLH.obj
 0002:00000f38       ??_C@_0BP@CHJPNNEM@JVMTI_ERROR_ABSENT_INFORMATION@ 0000000180004f38     libredefineCFLH.obj
 0002:00000f58       ??_C@_0BP@OMFMNLC@JVMTI_ERROR_INVALID_EVENT_TYPE@ 0000000180004f58     libredefineCFLH.obj
 0002:00000f78       ??_C@_0BN@BIBNPHHO@JVMTI_ERROR_ILLEGAL_ARGUMENT@ 0000000180004f78     libredefineCFLH.obj
 0002:00000f98       ??_C@_0BK@KKNDHDCE@JVMTI_ERROR_NATIVE_METHOD@ 0000000180004f98     libredefineCFLH.obj
 0002:00000fb8       ??_C@_0BK@PMKCFHAE@JVMTI_ERROR_OUT_OF_MEMORY@ 0000000180004fb8     libredefineCFLH.obj
 0002:00000fd8       ??_C@_0BK@NNJBDMNB@JVMTI_ERROR_ACCESS_DENIED@ 0000000180004fd8     libredefineCFLH.obj
 0002:00000ff8       ??_C@_0BI@GHECLMNC@JVMTI_ERROR_WRONG_PHASE@ 0000000180004ff8     libredefineCFLH.obj
 0002:00001010       ??_C@_0BF@OLIHJOII@JVMTI_ERROR_INTERNAL@ 0000000180005010     libredefineCFLH.obj
 0002:00001028       ??_C@_0BO@EOHGKJHI@JVMTI_ERROR_UNATTACHED_THREAD@ 0000000180005028     libredefineCFLH.obj
 0002:00001048       ??_C@_0CA@LKHFDACL@JVMTI_ERROR_INVALID_ENVIRONMENT@ 0000000180005048     libredefineCFLH.obj
 0002:00001068       ??_C@_0BA@MMFHLOKK@?$DMunknown?5error?$DO@ 0000000180005068     libredefineCFLH.obj
 0002:00001078       ??_C@_0CF@CBHOKDB@throwable?5?$DN?5jni?9?$DOExceptionOccur@ 0000000180005078     libredefineCFLH.obj
 0002:000010a0       ??_C@_03OFAPEBGM@?$CFs?6@  00000001800050a0     libredefineCFLH.obj
 0002:000010a8       ??_C@_0DM@LPIGEGNJ@s?2test?2hotspot?2jtreg?2vmTestbase@ 00000001800050a8     libredefineCFLH.obj
 0002:000010e8       ??_C@_0CC@NFCNPEPK@Exception?5in?5JNI?5call?5?$CIcleared?$CJ@ 00000001800050e8     libredefineCFLH.obj
 0002:00001110       ??_C@_0BJ@IBAKFIKF@jni?9?$DOExceptionDescribe?$CI?$CJ@ 0000000180005110     libredefineCFLH.obj
 0002:00001130       ??_C@_0BG@GGKALKMH@jni?9?$DOExceptionClear?$CI?$CJ@ 0000000180005130     libredefineCFLH.obj
 0002:00001148       ??_C@_0CF@JMGFGJLJ@?$CD?5?5?5verified?5JNI?5assertion?5is?5F@ 0000000180005148     libredefineCFLH.obj
 0002:00001170       ??_C@_0CB@MLNJNCLJ@?5?5jvmti?5error?3?5code?$DN?$CFd?0?5name?$DN?$CFs@ 0000000180005170     libredefineCFLH.obj
 0002:00001198       ??_C@_0CD@OHBGDKMK@?$CD?5?5?5jvmti?5error?3?5code?$DN?$CFd?0?5name?$DN@ 0000000180005198     libredefineCFLH.obj
 0002:000011c0       ??_C@_0CG@JNNCGPHB@?$CD?5?5?5error?5expected?3?5code?$DN?$CFd?0?5na@ 00000001800051c0     libredefineCFLH.obj
 0002:000011f0       ??_C@_0EB@IMGKPCGE@?$CIstr_obj?5?$DN?5jni?9?$DONewStringUTF?$CIco@ 00000001800051f0     libredefineCFLH.obj
 0002:00001240       ??_C@_0EA@HFOGGBCC@s?2test?2hotspot?2jtreg?2vmTestbase@ 0000000180005240     libredefineCFLH.obj
 0002:00001280       ??_C@_05KKCIMGE@error@     0000000180005280     libredefineCFLH.obj
 0002:00001290       ??_C@_0EA@PNBCDMOA@s?2test?2hotspot?2jtreg?2vmTestbase@ 0000000180005290     libredefineCFLH.obj
 0002:000012d0       ??_C@_0DI@ILAHDLMP@?$CI?$CKagentThreadProc?$CJ?$CIjvmti_env?0?5a@ 00000001800052d0     libredefineCFLH.obj
 0002:00001308       ??_C@_0BD@KDBALNLB@JVMTI?5agent?5thread@ 0000000180005308     libredefineCFLH.obj
 0002:00001320       ??_C@_0BB@NOKBFPFO@java?1lang?1Thread@ 0000000180005320     libredefineCFLH.obj
 0002:00001334       ??_C@_06FALKBLGB@?$DMinit?$DO@ 0000000180005334     libredefineCFLH.obj
 0002:00001340       ??_C@_0BG@IKDDPPGD@?$CILjava?1lang?1String?$DL?$CJV@ 0000000180005340     libredefineCFLH.obj
 0002:00001360       ??_C@_0EB@IFJBFEKC@?$CIthreadClass?5?$DN?5jni_env?9?$DOFindCla@ 0000000180005360     libredefineCFLH.obj
 0002:000013b0       ??_C@_0GF@FGFIBKKL@?$CIthreadCtor?5?$DN?5jni_env?9?$DOGetMetho@ 00000001800053b0     libredefineCFLH.obj
 0002:00001418       ??_C@_0DN@NCPDJLOG@?$CIthreadName?5?$DN?5jni_env?9?$DONewStrin@ 0000000180005418     libredefineCFLH.obj
 0002:00001460       ??_C@_0FE@PFKODBGC@?$CIthreadObject?5?$DN?5jni_env?9?$DONewObj@ 0000000180005460     libredefineCFLH.obj
 0002:000014c0       ??_C@_0ED@HOBAHHJI@?$CIthreadGlobalRef?5?$DN?5jni_env?9?$DONew@ 00000001800054c0     libredefineCFLH.obj
 0002:00001510       ??_C@_0FN@HNJJAHFC@jvmti_env?9?$DORunAgentThread?$CIagent@ 0000000180005510     libredefineCFLH.obj
 0002:00001570       ??_C@_0EA@MOJDNKDF@Debuggee?5status?5sync?5aborted?5be@ 0000000180005570     libredefineCFLH.obj
 0002:000015b0       ??_C@_0EA@EEOEJAEN@status?5?$DN?5syncDebuggeeStatus?$CIjni@ 00000001800055b0     libredefineCFLH.obj
 0002:000015f0       ??_C@_0BL@JBCFNBMB@nsk_jvmti_resetAgentData?$CI?$CJ@ 00000001800055f0     libredefineCFLH.obj
 0002:00001610       ??_C@_0EL@LPBEELIP@s?2test?2hotspot?2jtreg?2vmTestbase@ 0000000180005610     libredefineCFLH.obj
 0002:00001660       ??_C@_0CK@JDAMFDMJ@jvmti?9?$DOSetTag?$CIo?0?5tag?$CJ?5?$DN?$DN?5JVMTI_@ 0000000180005660     libredefineCFLH.obj
 0002:00001690       ??_C@_0CC@DAMNHKNI@Can?8t?5set?5tag?5?$CFli?5for?5object?5?$CFl@ 0000000180005690     libredefineCFLH.obj
 0002:000016b8       ??_C@_0DL@HAJPNKEF@jvmti?9?$DOGetObjectHashCode?$CIo?0?5?$CGha@ 00000001800056b8     libredefineCFLH.obj
 0002:000016f8       ??_C@_0BL@JFPIEOBF@Can?8t?5get?5hash?5object?5?$CFlx?6@ 00000001800056f8     libredefineCFLH.obj
 0002:00001718       ??_C@_0BG@DICPHBKN@setTag?3?5?$CF08x?5?$DM?9?5?$CF?53li@ 0000000180005718     libredefineCFLH.obj
 0002:00001730       ??_C@_0DH@FCEEBDMJ@?$CIs?5?$DN?5jni?9?$DOGetStringUTFChars?$CIsIn@ 0000000180005730     libredefineCFLH.obj
 0002:00001768       ??_C@_0BJ@OKKGHDCN@Can?8t?5get?5string?5at?5?$CF?$CDp?6@ 0000000180005768     libredefineCFLH.obj
 0002:00001788       ??_C@_0BP@EKFLGGFJ@Can?8t?5get?5string?5at?5?$CF?$CDp?3?5null?6@ 0000000180005788     libredefineCFLH.obj
 0002:000017a8       ??_C@_06ICODBHCL@?5?1?1?5?$CFs@ 00000001800057a8     libredefineCFLH.obj
 0002:000017b0       ??_C@_0DB@KGFPLEGO@?$CIr?5?$DN?5jvmti?9?$DOGetTag?$CIo?0?5?$CGtag?$CJ?$CJ?5?$DN?$DN@ 00000001800057b0     libredefineCFLH.obj
 0002:000017e8       ??_C@_0CO@PDAGBCGJ@Can?8t?5GetTag?5for?5object?5?$CFlx?4?5Re@ 00000001800057e8     libredefineCFLH.obj
 0002:00001818       ??_C@_0CH@HPEODOHC@TEST_BUG?3?5Max?4?5number?5of?5refs?5r@ 0000000180005818     libredefineCFLH.obj
 0002:00001840       ??_C@_0DI@PHFCABIM@?$CIr?5?$DN?5jvmti?9?$DOGetTag?$CIfrom?0?5?$CGtagFr@ 0000000180005840     libredefineCFLH.obj
 0002:00001878       ??_C@_0DI@MDEGFNKD@TEST_BUG?3?5Can?8t?5GetTag?5for?5obje@ 0000000180005878     libredefineCFLH.obj
 0002:000018b0       ??_C@_0DE@MLELJAHM@?$CIr?5?$DN?5jvmti?9?$DOGetTag?$CIto?0?5?$CGtagTo?$CJ?$CJ@ 00000001800058b0     libredefineCFLH.obj
 0002:000018e8       ??_C@_0BH@MEDHAAFL@VMInit?5event?5received?6@ 00000001800058e8     libredefineCFLH.obj
 0002:00001900       ??_C@_0DC@ILIOKICC@Received?5class?5file?5load?5hook?5e@ 0000000180005900     libredefineCFLH.obj
 0002:00001938       ??_C@_0CP@HMGAFMHE@?$CIGetClassSignature?$CJ?5unexpected?5@ 0000000180005938     libredefineCFLH.obj
 0002:00001968       ??_C@_0CG@NIPDKNBE@redefined?5class?5name?5signature?5@ 0000000180005968     libredefineCFLH.obj
 0002:00001990       ??_C@_0CG@NOPJCADI@?$CIAllocate?$CJ?5unexpected?5error?3?5?$CFs@ 0000000180005990     libredefineCFLH.obj
 0002:000019b8       ??_C@_09OPJEJKBL@printdump@ 00000001800059b8     libredefineCFLH.obj
 0002:000019d0       ??_C@_0FL@KBBIEGMD@s?2test?2hotspot?2jtreg?2vmTestbase@ 00000001800059d0     libredefineCFLH.obj
 0002:00001a30       ??_C@_0CF@JMMADLFE@?$CFs?3?5Failed?5to?5call?5GetEnv?3?5erro@ 0000000180005a30     libredefineCFLH.obj
 0002:00001a58       ??_C@_0DG@LAJPGIIE@?$CIGetPotentialCapabilities?$CJ?5unex@ 0000000180005a58     libredefineCFLH.obj
 0002:00001a90       ??_C@_0CN@LKPEOJPO@?$CIAddCapabilities?$CJ?5unexpected?5er@ 0000000180005a90     libredefineCFLH.obj
 0002:00001ac0       ??_C@_0CN@BCCBOHCH@?$CIGetCapabilities?$CJ?5unexpected?5er@ 0000000180005ac0     libredefineCFLH.obj
 0002:00001af0       ??_C@_0CN@DLBMMHNI@Warning?3?5RedefineClasses?5is?5not@ 0000000180005af0     libredefineCFLH.obj
 0002:00001b20       ??_C@_0CP@IMINGNLL@?$CISetEventCallbacks?$CJ?5unexpected?5@ 0000000180005b20     libredefineCFLH.obj
 0002:00001b50       ??_C@_0DF@GIHGOFNC@Failed?5to?5enable?5event?5JVMTI_EV@ 0000000180005b50     libredefineCFLH.obj
 0002:00001b90       ??_C@_0EC@FEFKBICJ@Failed?5to?5enable?5event?5JVMTI_EV@ 0000000180005b90     libredefineCFLH.obj
 0002:00001bd8       ??_C@_0CH@CDOJMNAO@JVMTI?5client?5was?5not?5properly?5l@ 0000000180005bd8     libredefineCFLH.obj
 0002:00001c00       ??_C@_0CE@OEKLHMDO@?$DO?$DO?$DO?$DO?$DO?$DO?$DO?$DO?5Invoke?5RedefineClasses@ 0000000180005c00     libredefineCFLH.obj
 0002:00001c28       ??_C@_0BK@LCHPJIGO@?7new?5class?5byte?5count?$DN?$CFd?6@ 0000000180005c28     libredefineCFLH.obj
 0002:00001c48       ??_C@_0CH@COFNDGGE@?$CFs?3?5Failed?5to?5call?5RedefineClas@ 0000000180005c48     libredefineCFLH.obj
 0002:00001c70       ??_C@_0CF@MKKOLKFO@?7the?5function?5returned?5error?5?$CFd@ 0000000180005c70     libredefineCFLH.obj
 0002:00001c98       ??_C@_0DF@KIBMOCOK@?7For?5more?5info?5about?5this?5error@ 0000000180005c98     libredefineCFLH.obj
 0002:00001cd0       ??_C@_0DB@JBFCAFBM@?$DM?$DM?$DM?$DM?$DM?$DM?$DM?$DM?5RedefineClasses?$CI?$CJ?5is?5s@ 0000000180005cd0     libredefineCFLH.obj
 0002:00001d20       ??_C@_1EC@JIJBPKFM@?$AAa?$AAp?$AAi?$AA?9?$AAm?$AAs?$AA?9?$AAw?$AAi?$AAn?$AA?9?$AAc?$AAo?$AAr?$AAe@ 0000000180005d20     MSVCRT:thread_safe_statics.obj
 0002:00001d68       ??_C@_1BK@MGMFAEKH@?$AAk?$AAe?$AAr?$AAn?$AAe?$AAl?$AA3?$AA2?$AA?4?$AAd?$AAl?$AAl@ 0000000180005d68     MSVCRT:thread_safe_statics.obj
 0002:00001d88       ??_C@_0BJ@JEBJOJFJ@SleepConditionVariableCS@ 0000000180005d88     MSVCRT:thread_safe_statics.obj
 0002:00001da8       ??_C@_0BJ@PGPPEPCC@WakeAllConditionVariable@ 0000000180005da8     MSVCRT:thread_safe_statics.obj
 0002:00001dc8       _pDefaultRawDllMain        0000000180005dc8     MSVCRT:dll_dllmain.obj
 0002:00001dc8       _pRawDllMain               0000000180005dc8     MSVCRT:dll_dllmain.obj
 0002:00001dd0       __xmm@ffffffffffffffffffffffffffffffff 0000000180005dd0     MSVCRT:utility.obj
 0002:00001de0       _load_config_used          0000000180005de0     MSVCRT:loadcfg.obj
 0002:00002000       _tls_used                  0000000180006000     MSVCRT:tlssup.obj
 0002:00002028       __volatile_metadata        0000000180006028     <linker-defined>
 0002:000023f8       __rtc_iaa                  00000001800063f8     MSVCRT:initsect.obj
 0002:00002400       __rtc_izz                  0000000180006400     MSVCRT:initsect.obj
 0002:00002408       __rtc_taa                  0000000180006408     MSVCRT:initsect.obj
 0002:00002410       __rtc_tzz                  0000000180006410     MSVCRT:initsect.obj
 0002:00002418       _tls_start                 0000000180006418     MSVCRT:tlssup.obj
 0002:0000241c       _Init_thread_epoch         000000018000641c     MSVCRT:thread_safe_statics.obj
 0002:00002420       _tls_end                   0000000180006420     MSVCRT:tlssup.obj
 0002:00002b08       __IMPORT_DESCRIPTOR_KERNEL32 0000000180006b08     kernel32:KERNEL32.dll
 0002:00002b1c       __IMPORT_DESCRIPTOR_VCRUNTIME140 0000000180006b1c     vcruntime:VCRUNTIME140.dll
 0002:00002b30       __IMPORT_DESCRIPTOR_api-ms-win-crt-runtime-l1-1-0 0000000180006b30     ucrt:api-ms-win-crt-runtime-l1-1-0.dll
 0002:00002b44       __IMPORT_DESCRIPTOR_api-ms-win-crt-stdio-l1-1-0 0000000180006b44     ucrt:api-ms-win-crt-stdio-l1-1-0.dll
 0002:00002b58       __IMPORT_DESCRIPTOR_api-ms-win-crt-string-l1-1-0 0000000180006b58     ucrt:api-ms-win-crt-string-l1-1-0.dll
 0002:00002b6c       __NULL_IMPORT_DESCRIPTOR   0000000180006b6c     kernel32:KERNEL32.dll
 0003:00000000       CLASS_NAME                 0000000180008000     libredefineCFLH.obj
 0003:00000038       _Init_global_epoch         0000000180008038     MSVCRT:thread_safe_statics.obj
 0003:00000040       __security_cookie          0000000180008040     MSVCRT:gs_cookie.obj
 0003:00000048       __security_cookie_complement 0000000180008048     MSVCRT:gs_cookie.obj
 0003:00000050       __scrt_native_dllmain_reason 0000000180008050     MSVCRT:utility.obj
 0003:00000058       __isa_available            0000000180008058     MSVCRT:cpu_disp.obj
 0003:0000005c       __isa_enabled              000000018000805c     MSVCRT:cpu_disp.obj
 0003:00000060       __memset_fast_string_threshold 0000000180008060     MSVCRT:cpu_disp.obj
 0003:00000068       __memset_nt_threshold      0000000180008068     MSVCRT:cpu_disp.obj
 0003:00000070       __scrt_ucrt_dll_is_in_use  0000000180008070     MSVCRT:ucrt_stubs.obj
 0003:00000080       g_wrongHeapCallbacks       0000000180008080     libredefineCFLH.obj
 0003:00000100       g_szTagInfo                0000000180008100     libredefineCFLH.obj
 0003:00002040       g_tagFlags                 000000018000a040     libredefineCFLH.obj
 0003:00002428       g_refsToVerifyCnt          000000018000a428     libredefineCFLH.obj
 0003:0000242c       g_fakeUserData             000000018000a42c     libredefineCFLH.obj
 0003:00002430       g_tagVisitCount            000000018000a430     libredefineCFLH.obj
 0003:000033d0       g_refsToVerify             000000018000b3d0     libredefineCFLH.obj
 0003:0001aad0       g_userDataError            0000000180022ad0     libredefineCFLH.obj
 0003:0001adb8       ?_OptionsStorage@?1??__local_stdio_printf_options@@9@4_KA 0000000180022db8     libredefineCFLH.obj
 0003:0001b378       _tls_index                 0000000180023378     MSVCRT:tlssup.obj
 0003:0001b380       __scrt_current_native_startup_state 0000000180023380     MSVCRT:utility.obj
 0003:0001b388       __scrt_native_startup_lock 0000000180023388     MSVCRT:utility.obj
 0003:0001b3c8       __scrt_debugger_hook_flag  00000001800233c8     MSVCRT:utility_desktop.obj
 0003:0001b3d0       ?__type_info_root_node@@3U__type_info_node@@A 00000001800233d0     MSVCRT:tncleanup.obj
 0003:0001b3e0       ?_OptionsStorage@?1??__local_stdio_scanf_options@@9@4_KA 00000001800233e0     MSVCRT:default_local_stdio_options.obj
 0003:0001b3e8       __favor                    00000001800233e8     MSVCRT:cpu_disp.obj
 0003:0001b3f0       __dyn_tls_init_callback    00000001800233f0     <common>

 entry point at        0001:00002410

 Static symbols

 0000:fffda000       .debug$S                   0000000180000000     redefineCFLH.exp
 0000:fffda000       .debug$S                   0000000180000000     vcruntime:VCRUNTIME140.dll
 0000:fffda000       .debug$S                   0000000180000000     vcruntime:VCRUNTIME140.dll
 0000:fffda000       .debug$S                   0000000180000000     vcruntime:VCRUNTIME140.dll
 0000:fffda000       .debug$S                   0000000180000000     vcruntime:VCRUNTIME140.dll
 0000:fffda000       .debug$S                   0000000180000000     vcruntime:VCRUNTIME140.dll
 0000:fffda000       .debug$S                   0000000180000000     vcruntime:VCRUNTIME140.dll
 0000:fffda000       .debug$S                   0000000180000000     vcruntime:VCRUNTIME140.dll
 0000:fffda000       .debug$S                   0000000180000000     ucrt:api-ms-win-crt-convert-l1-1-0.dll
 0002:ffffc000       .idata$6                   0000000180000000     ucrt:api-ms-win-crt-convert-l1-1-0.dll
 0000:fffda000       .debug$S                   0000000180000000     ucrt:api-ms-win-crt-heap-l1-1-0.dll
 0000:fffda000       .debug$S                   0000000180000000     ucrt:api-ms-win-crt-heap-l1-1-0.dll
 0000:fffda000       .debug$S                   0000000180000000     ucrt:api-ms-win-crt-heap-l1-1-0.dll
 0000:fffda000       .debug$S                   0000000180000000     ucrt:api-ms-win-crt-heap-l1-1-0.dll
 0002:ffffc000       .idata$6                   0000000180000000     ucrt:api-ms-win-crt-heap-l1-1-0.dll
 0000:fffda000       .debug$S                   0000000180000000     ucrt:api-ms-win-crt-runtime-l1-1-0.dll
 0000:fffda000       .debug$S                   0000000180000000     ucrt:api-ms-win-crt-runtime-l1-1-0.dll
 0000:fffda000       .debug$S                   0000000180000000     ucrt:api-ms-win-crt-runtime-l1-1-0.dll
 0000:fffda000       .debug$S                   0000000180000000     ucrt:api-ms-win-crt-runtime-l1-1-0.dll
 0000:fffda000       .debug$S                   0000000180000000     ucrt:api-ms-win-crt-runtime-l1-1-0.dll
 0000:fffda000       .debug$S                   0000000180000000     ucrt:api-ms-win-crt-runtime-l1-1-0.dll
 0000:fffda000       .debug$S                   0000000180000000     ucrt:api-ms-win-crt-runtime-l1-1-0.dll
 0000:fffda000       .debug$S                   0000000180000000     ucrt:api-ms-win-crt-runtime-l1-1-0.dll
 0000:fffda000       .debug$S                   0000000180000000     ucrt:api-ms-win-crt-runtime-l1-1-0.dll
 0000:fffda000       .debug$S                   0000000180000000     ucrt:api-ms-win-crt-runtime-l1-1-0.dll
 0000:fffda000       .debug$S                   0000000180000000     ucrt:api-ms-win-crt-runtime-l1-1-0.dll
 0000:fffda000       .debug$S                   0000000180000000     ucrt:api-ms-win-crt-runtime-l1-1-0.dll
 0000:fffda000       .debug$S                   0000000180000000     ucrt:api-ms-win-crt-runtime-l1-1-0.dll
 0000:fffda000       .debug$S                   0000000180000000     ucrt:api-ms-win-crt-runtime-l1-1-0.dll
 0000:fffda000       .debug$S                   0000000180000000     ucrt:api-ms-win-crt-runtime-l1-1-0.dll
 0000:fffda000       .debug$S                   0000000180000000     ucrt:api-ms-win-crt-runtime-l1-1-0.dll
 0000:fffda000       .debug$S                   0000000180000000     ucrt:api-ms-win-crt-stdio-l1-1-0.dll
 0000:fffda000       .debug$S                   0000000180000000     ucrt:api-ms-win-crt-stdio-l1-1-0.dll
 0000:fffda000       .debug$S                   0000000180000000     ucrt:api-ms-win-crt-stdio-l1-1-0.dll
 0000:fffda000       .debug$S                   0000000180000000     ucrt:api-ms-win-crt-stdio-l1-1-0.dll
 0000:fffda000       .debug$S                   0000000180000000     ucrt:api-ms-win-crt-stdio-l1-1-0.dll
 0000:fffda000       .debug$S                   0000000180000000     ucrt:api-ms-win-crt-stdio-l1-1-0.dll
 0000:fffda000       .debug$S                   0000000180000000     ucrt:api-ms-win-crt-stdio-l1-1-0.dll
 0000:fffda000       .debug$S                   0000000180000000     ucrt:api-ms-win-crt-stdio-l1-1-0.dll
 0000:fffda000       .debug$S                   0000000180000000     ucrt:api-ms-win-crt-stdio-l1-1-0.dll
 0000:fffda000       .debug$S                   0000000180000000     ucrt:api-ms-win-crt-stdio-l1-1-0.dll
 0000:fffda000       .debug$S                   0000000180000000     ucrt:api-ms-win-crt-string-l1-1-0.dll
 0000:fffda000       .debug$S                   0000000180000000     ucrt:api-ms-win-crt-string-l1-1-0.dll
 0000:fffda000       .debug$S                   0000000180000000     ucrt:api-ms-win-crt-string-l1-1-0.dll
 0000:fffda000       .debug$S                   0000000180000000     ucrt:api-ms-win-crt-string-l1-1-0.dll
 0000:fffda000       .debug$S                   0000000180000000     ucrt:api-ms-win-crt-string-l1-1-0.dll
 0000:fffda000       .debug$S                   0000000180000000     ucrt:api-ms-win-crt-string-l1-1-0.dll
 0000:fffda000       .debug$S                   0000000180000000     ucrt:api-ms-win-crt-string-l1-1-0.dll
 0000:fffda000       .debug$S                   0000000180000000     ucrt:api-ms-win-crt-string-l1-1-0.dll
 0000:fffda000       .debug$S                   0000000180000000     kernel32:KERNEL32.dll
 0000:fffda000       .debug$S                   0000000180000000     kernel32:KERNEL32.dll
 0000:fffda000       .debug$S                   0000000180000000     kernel32:KERNEL32.dll
 0000:fffda000       .debug$S                   0000000180000000     kernel32:KERNEL32.dll
 0000:fffda000       .debug$S                   0000000180000000     kernel32:KERNEL32.dll
 0000:fffda000       .debug$S                   0000000180000000     kernel32:KERNEL32.dll
 0000:fffda000       .debug$S                   0000000180000000     kernel32:KERNEL32.dll
 0000:fffda000       .debug$S                   0000000180000000     kernel32:KERNEL32.dll
 0000:fffda000       .debug$S                   0000000180000000     kernel32:KERNEL32.dll
 0000:fffda000       .debug$S                   0000000180000000     kernel32:KERNEL32.dll
 0000:fffda000       .debug$S                   0000000180000000     kernel32:KERNEL32.dll
 0000:fffda000       .debug$S                   0000000180000000     kernel32:KERNEL32.dll
 0000:fffda000       .debug$S                   0000000180000000     kernel32:KERNEL32.dll
 0000:fffda000       .debug$S                   0000000180000000     kernel32:KERNEL32.dll
 0000:fffda000       .debug$S                   0000000180000000     kernel32:KERNEL32.dll
 0000:fffda000       .debug$S                   0000000180000000     kernel32:KERNEL32.dll
 0000:fffda000       .debug$S                   0000000180000000     kernel32:KERNEL32.dll
 0000:fffda000       .debug$S                   0000000180000000     kernel32:KERNEL32.dll
 0000:fffda000       .debug$S                   0000000180000000     kernel32:KERNEL32.dll
 0000:fffda000       .debug$S                   0000000180000000     kernel32:KERNEL32.dll
 0000:fffda000       .debug$S                   0000000180000000     kernel32:KERNEL32.dll
 0000:fffda000       .debug$S                   0000000180000000     kernel32:KERNEL32.dll
 0000:fffda000       .debug$S                   0000000180000000     kernel32:KERNEL32.dll
 0000:fffda000       .debug$S                   0000000180000000     kernel32:KERNEL32.dll
 0000:fffda000       .debug$S                   0000000180000000     kernel32:KERNEL32.dll
 0000:fffda000       .debug$S                   0000000180000000     kernel32:KERNEL32.dll
 0000:fffda000       .debug$S                   0000000180000000     kernel32:KERNEL32.dll
 0000:fffda000       .debug$S                   0000000180000000     kernel32:KERNEL32.dll
 0001:000010a4       addRefToVerify             00000001800020a4 f   libredefineCFLH.obj
 0001:00001118       agentThreadWrapper         0000000180002118 f   libredefineCFLH.obj
 0001:000012f0       file_basename              00000001800022f0 f   libredefineCFLH.obj
 0001:00001918       startAgentThreadWrapper    0000000180002918 f   libredefineCFLH.obj
 0001:00001c44       syncDebuggeeStatus         0000000180002c44 f   libredefineCFLH.obj
 0001:00001ecc       capture_previous_context   0000000180002ecc f   MSVCRT:gs_report.obj
 0001:00001f40       ?__scrt_initialize_thread_safe_statics@@YAHXZ 0000000180002f40 f   MSVCRT:thread_safe_statics.obj
 0001:00002010       ?__scrt_uninitialize_thread_safe_statics@@YAXXZ 0000000180003010 f   MSVCRT:thread_safe_statics.obj
 0001:000020c0       $$000000                   00000001800030c0     MSVCRT:amdsecgs.obj
 0001:000020f0       ?dllmain_crt_dispatch@@YAHQEAUHINSTANCE__@@KQEAX@Z 00000001800030f0 f   MSVCRT:dll_dllmain.obj
 0001:00002140       ?dllmain_crt_process_attach@@YAHQEAUHINSTANCE__@@QEAX@Z 0000000180003140 f   MSVCRT:dll_dllmain.obj
 0001:00002258       ?dllmain_crt_process_detach@@YAH_N@Z 0000000180003258 f   MSVCRT:dll_dllmain.obj
 0001:000022dc       ?dllmain_dispatch@@YAHQEAUHINSTANCE__@@KQEAX@Z 00000001800032dc f   MSVCRT:dll_dllmain.obj
 0001:00002cf0       $$000000                   0000000180003cf0     MSVCRT:guard_dispatch.obj
 0001:00002d10       $$000000                   0000000180003d10     MSVCRT:guard_xfg_dispatch.obj
 0001:00002d26       ?fin$0@?0??dllmain_crt_process_attach@@YAHQEAUHINSTANCE__@@QEAX@Z@4HA 0000000180003d26 f   MSVCRT:dll_dllmain.obj
 0001:00002d3d       ?fin$0@?0??dllmain_crt_process_detach@@YAH_N@Z@4HA 0000000180003d3d f   MSVCRT:dll_dllmain.obj
 0001:00002d56       ?fin$1@?0??dllmain_crt_process_detach@@YAH_N@Z@4HA 0000000180003d56 f   MSVCRT:dll_dllmain.obj
 0001:00002d6a       ?filt$0@?0??dllmain_dispatch@@YAHQEAUHINSTANCE__@@KQEAX@Z@4HA 0000000180003d6a f   MSVCRT:dll_dllmain.obj
 0001:00002da0       __scrt_is_nonwritable_in_current_image$filt$0 0000000180003da0 f   MSVCRT:utility.obj
 0002:000001e8       ?__scrt_initialize_tss_var@@3P6AHXZEA 00000001800041e8     MSVCRT:thread_safe_statics.obj
 0002:00000310       ?opcLengths@@3QBEB         0000000180004310     libredefineCFLH.obj
 0002:00001d08       GS_ExceptionPointers       0000000180005d08     MSVCRT:gs_report.obj
 0002:00002428       $unwind$fprintf            0000000180006428     libredefineCFLH.obj
 0002:00002434       $unwind$printf             0000000180006434     libredefineCFLH.obj
 0002:00002440       $unwind$?NewObject@JNIEnv_@@QEAAPEAV_jobject@@PEAV_jclass@@PEAU_jmethodID@@ZZ 0000000180006440     libredefineCFLH.obj
 0002:00002440       $unwind$nsk_lcomplain      0000000180006440     libredefineCFLH.obj
 0002:00002440       $unwind$nsk_ldisplay       0000000180006440     libredefineCFLH.obj
 0002:00002448       $unwind$nsk_lvdisplay      0000000180006448     libredefineCFLH.obj
 0002:00002448       $unwind$_RTC_Initialize    0000000180006448     MSVCRT:initsect.obj
 0002:00002448       $unwind$_RTC_Terminate     0000000180006448     MSVCRT:initsect.obj
 0002:00002448       $unwind$?__scrt_initialize_thread_safe_statics@@YAHXZ 0000000180006448     MSVCRT:thread_safe_statics.obj
 0002:00002454       $unwind$nsk_lvcomplain     0000000180006454     libredefineCFLH.obj
 0002:0000246c       $unwind$nsk_ltrace         000000018000646c     libredefineCFLH.obj
 0002:0000246c       $unwind$__report_gsfailure 000000018000646c     MSVCRT:gs_report.obj
 0002:00002474       $unwind$nsk_lvtrace        0000000180006474     libredefineCFLH.obj
 0002:00002474       $unwind$__raise_securityfailure 0000000180006474     MSVCRT:gs_report.obj
 0002:00002474       $unwind$__scrt_initialize_crt 0000000180006474     MSVCRT:utility.obj
 0002:00002474       $unwind$__scrt_initialize_onexit_tables 0000000180006474     MSVCRT:utility.obj
 0002:00002474       $unwind$__scrt_release_startup_lock 0000000180006474     MSVCRT:utility.obj
 0002:00002474       $unwind$__scrt_uninitialize_crt 0000000180006474     MSVCRT:utility.obj
 0002:00002474       $unwind$_onexit            0000000180006474     MSVCRT:utility.obj
 0002:0000247c       $unwind$nsk_lverify        000000018000647c     libredefineCFLH.obj
 0002:0000248c       $unwind$nsk_vprintf        000000018000648c     libredefineCFLH.obj
 0002:0000249c       $unwind$nsk_printf         000000018000649c     libredefineCFLH.obj
 0002:000024a4       $unwind$?nsk_jni_lverify@@YAHHPEAUJNIEnv_@@HQEBDH1ZZ 00000001800064a4     libredefineCFLH.obj
 0002:000024b8       $unwind$?nsk_jni_check_exception@@YAHPEAUJNIEnv_@@QEBDH@Z 00000001800064b8     libredefineCFLH.obj
 0002:000024d4       $unwind$Java_nsk_jvmti_unit_FollowReferences_FollowRefObjects_resetTags 00000001800064d4     libredefineCFLH.obj
 0002:000024d4       $unwind$VMInit             00000001800064d4     libredefineCFLH.obj
 0002:000024d4       $unwind$addRefToVerify     00000001800064d4     libredefineCFLH.obj
 0002:000024d4       $unwind$nsk_jvmti_resetAgentData 00000001800064d4     libredefineCFLH.obj
 0002:000024d4       $unwind$__scrt_initialize_default_local_stdio_options 00000001800064d4     MSVCRT:default_local_stdio_options.obj
 0002:000024d4       $unwind$?dllmain_crt_dispatch@@YAHQEAUHINSTANCE__@@KQEAX@Z 00000001800064d4     MSVCRT:dll_dllmain.obj
 0002:000024d4       $unwind$DllMain            00000001800064d4     MSVCRT:dll_dllmain_stub.obj
 0002:000024d4       $unwind$__GSHandlerCheck   00000001800064d4     MSVCRT:gshandler.obj
 0002:000024d4       $unwind$?__scrt_uninitialize_thread_safe_statics@@YAXXZ 00000001800064d4     MSVCRT:thread_safe_statics.obj
 0002:000024d4       $unwind$__scrt_acquire_startup_lock 00000001800064d4     MSVCRT:utility.obj
 0002:000024d4       $unwind$__scrt_dllmain_after_initialize_c 00000001800064d4     MSVCRT:utility.obj
 0002:000024d4       $unwind$__scrt_dllmain_before_initialize_c 00000001800064d4     MSVCRT:utility.obj
 0002:000024d4       $unwind$__scrt_dllmain_crt_thread_attach 00000001800064d4     MSVCRT:utility.obj
 0002:000024d4       $unwind$__scrt_dllmain_crt_thread_detach 00000001800064d4     MSVCRT:utility.obj
 0002:000024d4       $unwind$__scrt_dllmain_uninitialize_c 00000001800064d4     MSVCRT:utility.obj
 0002:000024d4       $unwind$__scrt_dllmain_uninitialize_critical 00000001800064d4     MSVCRT:utility.obj
 0002:000024d4       $unwind$atexit             00000001800064d4     MSVCRT:utility.obj
 0002:000024dc       $unwind$nsk_jvmti_lverify  00000001800064dc     libredefineCFLH.obj
 0002:000024f0       $unwind$exitOnError        00000001800064f0     libredefineCFLH.obj
 0002:00002500       $unwind$Java_nsk_share_jvmti_ArgumentHandler_getAgentOptionsString 0000000180006500     libredefineCFLH.obj
 0002:00002514       $unwind$Java_nsk_jvmti_unit_FollowReferences_FollowRefObjects_getTag 0000000180006514     libredefineCFLH.obj
 0002:00002514       $unwind$Java_nsk_share_jvmti_DebugeeClass_checkStatus 0000000180006514     libredefineCFLH.obj
 0002:00002514       $unwind$agentThreadWrapper 0000000180006514     libredefineCFLH.obj
 0002:00002524       $unwind$startAgentThreadWrapper 0000000180006524     libredefineCFLH.obj
 0002:00002540       $unwind$syncDebuggeeStatus 0000000180006540     libredefineCFLH.obj
 0002:00002540       $unwind$__scrt_dllmain_exception_filter 0000000180006540     MSVCRT:utility.obj
 0002:00002554       $unwind$Java_nsk_share_jvmti_DebugeeClass_resetAgentData 0000000180006554     libredefineCFLH.obj
 0002:0000255c       $unwind$ClassFileLoadHook  000000018000655c     libredefineCFLH.obj
 0002:0000255c       $unwind$MA_checkStatus     000000018000655c     libredefineCFLH.obj
 0002:00002570       $unwind$Java_nsk_jvmti_unit_FollowReferences_FollowRefObjects_setTag 0000000180006570     libredefineCFLH.obj
 0002:00002588       $unwind$Java_nsk_jvmti_unit_FollowReferences_FollowRefObjects_addRefToVerify 0000000180006588     libredefineCFLH.obj
 0002:000025a4       $unwind$Agent_Initialize   00000001800065a4     libredefineCFLH.obj
 0002:000025b0       $unwind$Java_nsk_jvmti_unit_events_redefineCFLH_JvmtiTest_makeRedefinition 00000001800065b0     libredefineCFLH.obj
 0002:000025bc       $unwind$capture_previous_context 00000001800065bc     MSVCRT:gs_report.obj
 0002:000025c8       $unwind$__GSHandlerCheckCommon 00000001800065c8     MSVCRT:gshandler.obj
 0002:000025d0       $xdatasym                  00000001800065d0     MSVCRT:amdsecgs.obj
 0002:000025d4       $unwind$?dllmain_crt_process_attach@@YAHQEAUHINSTANCE__@@QEAX@Z 00000001800065d4     MSVCRT:dll_dllmain.obj
 0002:00002610       $unwind$?fin$0@?0??dllmain_crt_process_attach@@YAHQEAUHINSTANCE__@@QEAX@Z@4HA 0000000180006610     MSVCRT:dll_dllmain.obj
 0002:00002610       $unwind$?fin$0@?0??dllmain_crt_process_detach@@YAH_N@Z@4HA 0000000180006610     MSVCRT:dll_dllmain.obj
 0002:00002610       $unwind$?fin$1@?0??dllmain_crt_process_detach@@YAH_N@Z@4HA 0000000180006610     MSVCRT:dll_dllmain.obj
 0002:00002618       $unwind$?dllmain_crt_process_detach@@YAH_N@Z 0000000180006618     MSVCRT:dll_dllmain.obj
 0002:0000266c       $unwind$?dllmain_dispatch@@YAHQEAUHINSTANCE__@@KQEAX@Z 000000018000666c     MSVCRT:dll_dllmain.obj
 0002:00002694       $unwind$?filt$0@?0??dllmain_dispatch@@YAHQEAUHINSTANCE__@@KQEAX@Z@4HA 0000000180006694     MSVCRT:dll_dllmain.obj
 0002:0000269c       $unwind$_DllMainCRTStartup 000000018000669c     MSVCRT:dll_dllmain.obj
 0002:000026ac       $unwind$__scrt_is_nonwritable_in_current_image 00000001800066ac     MSVCRT:utility.obj
 0002:000026cc       $unwind$__scrt_is_nonwritable_in_current_image$filt$0 00000001800066cc     MSVCRT:utility.obj
 0002:000026d4       $unwind$__scrt_fastfail    00000001800066d4     MSVCRT:utility_desktop.obj
 0002:000026e4       $unwind$__security_init_cookie 00000001800066e4     MSVCRT:gs_support.obj
 0002:000026f0       $unwind$__isa_available_init 00000001800066f0     MSVCRT:cpu_disp.obj
 0002:00002700       $xdatasym                  0000000180006700     MSVCRT:guard_dispatch.obj
 0002:00002708       $xdatasym                  0000000180006708     MSVCRT:guard_xfg_dispatch.obj
 0002:00002710       .edata                     0000000180006710     redefineCFLH.exp
 0002:00002738       rgpv                       0000000180006738     redefineCFLH.exp
 0002:00002778       rgszName                   0000000180006778     redefineCFLH.exp
 0002:000027b8       rgwOrd                     00000001800067b8     redefineCFLH.exp
 0002:000027d8       szName                     00000001800067d8     redefineCFLH.exp
 0002:000027e9       $N00001                    00000001800067e9     redefineCFLH.exp
 0002:000027f8       $N00002                    00000001800067f8     redefineCFLH.exp
 0002:00002805       $N00003                    0000000180006805     redefineCFLH.exp
 0002:0000284a       $N00004                    000000018000684a     redefineCFLH.exp
 0002:00002887       $N00005                    0000000180006887     redefineCFLH.exp
 0002:000028cf       $N00006                    00000001800068cf     redefineCFLH.exp
 0002:0000290f       $N00007                    000000018000690f     redefineCFLH.exp
 0002:0000294c       $N00008                    000000018000694c     redefineCFLH.exp
 0002:00002988       $N00009                    0000000180006988     redefineCFLH.exp
 0002:000029cb       $N00010                    00000001800069cb     redefineCFLH.exp
 0002:00002a06       $N00011                    0000000180006a06     redefineCFLH.exp
 0002:00002a34       $N00012                    0000000180006a34     redefineCFLH.exp
 0002:00002a65       $N00013                    0000000180006a65     redefineCFLH.exp
 0002:00002a94       $N00014                    0000000180006a94     redefineCFLH.exp
 0002:00002ac3       $N00015                    0000000180006ac3     redefineCFLH.exp
 0002:00002af8       $N00016                    0000000180006af8     redefineCFLH.exp
 0002:00002f02       .idata$6                   0000000180006f02     kernel32:KERNEL32.dll
 0002:00002f66       .idata$6                   0000000180006f66     vcruntime:VCRUNTIME140.dll
 0002:000030d2       .idata$6                   00000001800070d2     ucrt:api-ms-win-crt-runtime-l1-1-0.dll
 0002:000030f4       .idata$6                   00000001800070f4     ucrt:api-ms-win-crt-stdio-l1-1-0.dll
 0002:00003114       .idata$6                   0000000180007114     ucrt:api-ms-win-crt-string-l1-1-0.dll
 0003:00000008       ?codeAttributeName@@3PEBDEB 0000000180008008     libredefineCFLH.obj
 0003:00000010       ?lineNumberAttributeName@@3PEBDEB 0000000180008010     libredefineCFLH.obj
 0003:00000018       ?localVarAttributeName@@3PEBDEB 0000000180008018     libredefineCFLH.obj
 0003:00000020       ?localVarTypeAttributeName@@3PEBDEB 0000000180008020     libredefineCFLH.obj
 0003:00000028       ?stackMapAttributeName@@3PEBDEB 0000000180008028     libredefineCFLH.obj
 0003:00000030       ?callBytes@@3PAEA          0000000180008030     libredefineCFLH.obj
 0003:00000034       ?allocBytes@@3PAEA         0000000180008034     libredefineCFLH.obj
 0003:0001aad4       redefineAttempted          0000000180022ad4     libredefineCFLH.obj
 0003:0001aad8       nsk_context                0000000180022ad8     libredefineCFLH.obj
 0003:0001aae4       redefineSucceed            0000000180022ae4     libredefineCFLH.obj
 0003:0001aae8       agentFailed                0000000180022ae8     libredefineCFLH.obj
 0003:0001aaec       currentAgentStatus         0000000180022aec     libredefineCFLH.obj
 0003:0001aaf0       context                    0000000180022af0     libredefineCFLH.obj
 0003:0001aba8       agentThread                0000000180022ba8     libredefineCFLH.obj
 0003:0001abb0       agentThreadProc            0000000180022bb0     libredefineCFLH.obj
 0003:0001abb8       agentThreadArg             0000000180022bb8     libredefineCFLH.obj
 0003:0001abc0       agent_data                 0000000180022bc0     libredefineCFLH.obj
 0003:0001abd0       jvmti_env                  0000000180022bd0     libredefineCFLH.obj
 0003:0001abd8       jvm                        0000000180022bd8     libredefineCFLH.obj
 0003:0001abe0       jni_env                    0000000180022be0     libredefineCFLH.obj
 0003:0001abe8       checkStatus_func           0000000180022be8     libredefineCFLH.obj
 0003:0001abf0       ?codeAttributeIndex@@3GA   0000000180022bf0     libredefineCFLH.obj
 0003:0001abf2       printdump                  0000000180022bf2     libredefineCFLH.obj
 0003:0001abf4       ?lineNumberAttributeIndex@@3GA 0000000180022bf4     libredefineCFLH.obj
 0003:0001abf8       ?localVarAttributeIndex@@3GA 0000000180022bf8     libredefineCFLH.obj
 0003:0001abfc       ?localVarTypeAttributeIndex@@3GA 0000000180022bfc     libredefineCFLH.obj
 0003:0001ac00       ?stackMapAttributeIndex@@3GA 0000000180022c00     libredefineCFLH.obj
 0003:0001ac04       ?stackFrameOffset@@3GA     0000000180022c04     libredefineCFLH.obj
 0003:0001ac08       ?mode@@3HA                 0000000180022c08     libredefineCFLH.obj
 0003:0001ac0c       ?constantPoolSize@@3GA     0000000180022c0c     libredefineCFLH.obj
 0003:0001ac10       ?orig@@3PEBEEB             0000000180022c10     libredefineCFLH.obj
 0003:0001ac18       ?gen@@3PEAEEA              0000000180022c18     libredefineCFLH.obj
 0003:0001ac20       ?inputPos@@3PEAEEA         0000000180022c20     libredefineCFLH.obj
 0003:0001ac28       ?endPos@@3PEBEEB           0000000180022c28     libredefineCFLH.obj
 0003:0001ac30       ?genPos@@3PEAEEA           0000000180022c30     libredefineCFLH.obj
 0003:0001ac38       ?markPos@@3PEAEEA          0000000180022c38     libredefineCFLH.obj
 0003:0001ac40       ?constantPool@@3PEAPEADEA  0000000180022c40     libredefineCFLH.obj
 0003:0001ac48       ?constantPoolCount@@3GA    0000000180022c48     libredefineCFLH.obj
 0003:0001ac4c       ?zeroBytes@@3PAEA          0000000180022c4c     libredefineCFLH.obj
 0003:0001ac50       ?codeLength@@3IA           0000000180022c50     libredefineCFLH.obj
 0003:0001ac54       result                     0000000180022c54     libredefineCFLH.obj
 0003:0001ac58       ?map@@3PEAIEA              0000000180022c58     libredefineCFLH.obj
 0003:0001ac60       ?widening@@3PEACEA         0000000180022c60     libredefineCFLH.obj
 0003:0001ac68       jvmti                      0000000180022c68     libredefineCFLH.obj
 0003:0001ac70       caps                       0000000180022c70     libredefineCFLH.obj
 0003:0001ac80       callbacks                  0000000180022c80     libredefineCFLH.obj
 0003:0001adc0       GS_ExceptionRecord         0000000180022dc0     MSVCRT:gs_report.obj
 0003:0001ae60       GS_ContextRecord           0000000180022e60     MSVCRT:gs_report.obj
 0003:0001b330       ?g_tss_cv@@3U_RTL_CONDITION_VARIABLE@@A 0000000180023330     MSVCRT:thread_safe_statics.obj
 0003:0001b338       ?g_tss_event@@3PEAXEA      0000000180023338     MSVCRT:thread_safe_statics.obj
 0003:0001b340       ?g_tss_mutex@@3U_RTL_CRITICAL_SECTION@@A 0000000180023340     MSVCRT:thread_safe_statics.obj
 0003:0001b368       ?g_sleep_condition_variable_cs@@3P6AHPEAU_RTL_CONDITION_VARIABLE@@PEAU_RTL_CRITICAL_SECTION@@K@ZEA 0000000180023368     MSVCRT:thread_safe_statics.obj
 0003:0001b370       ?g_wake_all_condition_variable@@3P6AXPEAU_RTL_CONDITION_VARIABLE@@@ZEA 0000000180023370     MSVCRT:thread_safe_statics.obj
 0003:0001b37c       ?__proc_attached@@3HA      000000018002337c     MSVCRT:dll_dllmain.obj
 0003:0001b390       ?is_initialized_as_dll@@3_NA 0000000180023390     MSVCRT:utility.obj
 0003:0001b391       ?module_local_atexit_table_initialized@@3_NA 0000000180023391     MSVCRT:utility.obj
 0003:0001b398       ?module_local_atexit_table@@3U_onexit_table_t@@A 0000000180023398     MSVCRT:utility.obj
 0003:0001b3b0       ?module_local_at_quick_exit_table@@3U_onexit_table_t@@A 00000001800233b0     MSVCRT:utility.obj
